:020000040800F2
:1000000000070020F5040008552D00080D2D0008FC
:10001000352D00080D2D00082D2D0008F7040008CF
:10002000F7040008F7040008F7040008253D00085D
:10003000F7040008F7040008F7040008F7040008B4
:10004000F7040008F7040008F7040008F7040008A4
:10005000F7040008F704000899500008C150000890
:10006000E95000081151000839510008F704000850
:10007000F7040008F7040008F7040008F704000874
:10008000F7040008F7040008F7040008F704000864
:10009000F7040008BD2C0008D12C000861510008AD
:1000A000F7040008F7040008F7040008F704000844
:1000B00049520008F7040008F7040008F704000894
:1000C000F7040008F7040008F7040008F704000824
:1000D000F7040008F704000835520008F704000888
:1000E000C5510008F7040008F7040008F7040008E9
:1000F000F7040008F7040008F7040008F7040008F4
:10010000F7040008F7040008F7040008F7040008E3
:10011000F7040008F7040008F7040008F7040008D3
:10012000F7040008F7040008F7040008F7040008C3
:10013000F7040008F7040008F7040008F7040008B3
:10014000F7040008F7040008F7040008F7040008A3
:10015000F7040008F7040008F7040008F704000893
:10016000F7040008F7040008F7040008F704000883
:10017000F7040008F7040008F7040008F704000873
:10018000F7040008F7040008F7040008F704000863
:10019000F7040008F7040008E52C0008F92C000813
:1001A000F7040008F7040008F7040008F704000843
:1001B000F7040008F7040008F7040008F704000833
:1001C000F7040008F7040008F7040008F704000823
:1001D000F7040008F7040008F7040008F704000813
:1001E000D116000800000000000000000000000020
:1001F00053B94AB9002908BF00281CBF4FF0FF318E
:100200004FF0FF3000F074B9ADF1080C6DE904CE89
:1002100000F006F8DDF804E0DDE9022304B07047E1
:100220002DE9F047089D04468E46002B4DD18A42A9
:10023000944669D9B2FA82F252B101FA02F3C2F1DC
:10024000200120FA01F10CFA02FC41EA030E94406D
:100250004FEA1C48210CBEFBF8F61FFA8CF708FB8E
:1002600016E341EA034306FB07F199420AD91CEB66
:10027000030306F1FF3080F01F81994240F21C8198
:10028000023E63445B1AA4B2B3FBF8F008FB1033E0
:1002900044EA034400FB07F7A7420AD91CEB040415
:1002A00000F1FF3380F00A81A74240F207816444E5
:1002B000023840EA0640E41B00261DB1D44000236A
:1002C000C5E900433146BDE8F0878B4209D9002DCE
:1002D00000F0EF800026C5E9000130463146BDE858
:1002E000F087B3FA83F6002E4AD18B4202D38242C2
:1002F00000F2F980841A61EB030301209E46002D71
:10030000E0D0C5E9004EDDE702B9FFDEB2FA82F2C5
:10031000002A40F09280A1EB0C014FEA1C471FFA23
:100320008CFE0126200CB1FBF7F307FB131140EA0A
:1003300001410EFB03F0884208D91CEB010103F1D7
:10034000FF3802D2884200F2CB804346091AA4B299
:10035000B1FBF7F007FB101144EA01440EFB00FE6D
:10036000A64508D91CEB040400F1FF3102D2A645D2
:1003700000F2BB800846A4EB0E0440EA03409CE771
:10038000C6F12007B34022FA07FC4CEA030C20FA1E
:1003900007F401FA06F31C43F9404FEA1C4900FA3E
:1003A00006F3B1FBF9F8200C1FFA8CFE09FB1811BB
:1003B00040EA014108FB0EF0884202FA06F20BD92E
:1003C0001CEB010108F1FF3A80F08880884240F27E
:1003D0008580A8F102086144091AA4B2B1FBF9F0C2
:1003E00009FB101144EA014100FB0EFE8E4508D9BD
:1003F0001CEB010100F1FF346CD28E456AD9023842
:10040000614440EA0840A0FB0294A1EB0E01A14226
:10041000C846A64656D353D05DB1B3EB080261EB94
:100420000E0101FA07F722FA06F3F1401F43C5E96E
:10043000007100263146BDE8F087C2F12003D840A4
:100440000CFA02FC21FA03F3914001434FEA1C47E6
:100450001FFA8CFEB3FBF7F007FB10360B0C43EAD8
:10046000064300FB0EF69E4204FA02F408D91CEB88
:10047000030300F1FF382FD29E422DD90238634486
:100480009B1B89B2B3FBF7F607FB163341EA034126
:1004900006FB0EF38B4208D91CEB010106F1FF3875
:1004A00016D28B4214D9023E6144C91A46EA00466C
:1004B00038E72E46284605E70646E3E61846F8E6FE
:1004C0004B45A9D2B9EB020864EB0C0E0138A3E747
:1004D0004646EAE7204694E74046D1E7D0467BE728
:1004E000023B614432E7304609E76444023842E7A0
:1004F000704700BF02E000F000F8FEE772B6374830
:1005000080F30888364880F3098836483649086001
:1005100040F20000CCF200004EF63471CEF2000141
:100520000860BFF34F8FBFF36F8F40F20000C0F23F
:10053000F0004EF68851CEF200010860BFF34F8FF5
:10054000BFF36F8F4FF00000E1EE100A4EF63C71E2
:10055000CEF200010860062080F31488BFF36F8F8D
:1005600004F0CAFB04F05CFC4FF055301F491B4AF5
:1005700091423CBF41F8040BFAE71D49184A9142E9
:100580003CBF41F8040BFAE71A491B4A1B4B9A423D
:100590003EBF51F8040B42F8040BF8E7002018495D
:1005A000184A91423CBF41F8040BFAE704F0A8FB5B
:1005B00004F07CFC144C154DAC4203DA54F8041BD7
:1005C0008847F9E700F042F8114C124DAC4203DACB
:1005D00054F8041B8847F9E704F090BB000700209B
:1005E000002300200000000808ED00E000010020CA
:1005F0000007002060550008002300208C23002005
:100600009023002028650020E0010008E401000894
:10061000E4010008E40100082DE9F04F2DED108AF7
:10062000C1F80CD0C3689D46BDEC108ABDE8F08FC0
:10063000002383F311882846A047002003F0D8FF49
:10064000FEE703F03BFF00DFFEE70000F8B504F033
:10065000F5FA074604F046FB0546B8BB204B9F421F
:1006600034D001339F4234D01E4B27F0FF029A4210
:1006700032D1F8B200F052FE2E4642F2107400F071
:1006800053FE08B10024264601F0D6FA20B103201B
:1006900000F07CF80024264635B1134B9F4203D06E
:1006A00004F018FB00242646002004F0D1FA0EB115
:1006B00000F082F801F08AF900F05AFE01F07AF8B1
:1006C000204600F0D1F800F077F8F9E72E46002434
:1006D000D5E704460126D2E7064640F6C414CEE725
:1006E000010007B0000008B0263A09B008B501F0D3
:1006F0002DF8A0F120035842584108BD07B541F23A
:100700001203022101A8ADF8043001F03DF803B056
:100710005DF804FB38B5302383F31188174803686C
:100720000BB104F023F8164A144800234FF47A71F1
:1007300004F012F8002383F31188124C236813B1DC
:100740002368013B2360636813B16368013B636006
:100750000D4D2B7833B963687BB9022001F0C4F8E2
:10076000322363602B78032B07D163682BB90220F7
:1007700001F0BAF84FF47A73636038BD902300201B
:1007800015070008B0240020A8230020084B18708B
:1007900003280CD8DFE800F008050208022001F069
:1007A00099B8022001F08CB8024B00225A607047C1
:1007B000A8230020B024002010B501F03DFA30B18C
:1007C000234B03221A70234B00225A6010BD224B88
:1007D000224A1C4619680131F8D004339342F9D1FA
:1007E0006268A242F2D31E4B9B6803F1006303F5DB
:1007F00010439A42EAD204F03FFA04F051FA002082
:1008000000F0F2FF0220FFF7C1FF164B9A6D0022A5
:100810009A65996F9A67996FD96DDA65D96FDA67BA
:10082000D96F196E1A66D3F88010C3F88020D3F8F8
:10083000803072B64FF0E0233021C3F8084DD4E980
:10084000003281F311889D4683F308881047BDE785
:10085000A8230020B0240020009000082090000869
:1008600000230020001002402DE9F04F93B0AC4B64
:1008700000902022FF210AA89D6801F051F8A94AA2
:100880001378A3B9A848012103601170302383F3C2
:10089000118803680BB103F069FFA44AA248002342
:1008A0004FF47A7103F058FF002383F31188009B03
:1008B00013B19F4B009A1A609E4A009C1378032B39
:1008C0001EBF002313709A4A4FF0000A18BF5360EE
:1008D000D3465646D146012000F0FCFF24B1944B8C
:1008E0001B68002B00F01582002000F02FFF039002
:1008F000039B002B01DA00F08FFD039B002BEDDB47
:10090000012000F0DDFF039B213B162BE3D801A261
:1009100052F823F071090008990900082D0A00080F
:10092000D7080008D7080008D7080008B70A000849
:10093000870C0008A10B0008030C00082B0C000812
:10094000510C0008D7080008630C0008D7080008FD
:10095000D50C0008110A0008D7080008190D000876
:100960007D090008110A0008D7080008030C0008D8
:100970000220FFF7BBFE002840F0F581009B02211A
:10098000BAF1000F08BF1C4605A841F21233ADF8BA
:10099000143000F0F9FE9EE74FF47A7000F0D6FEB6
:1009A000071EEBDB0220FFF7A1FE0028E6D0013F87
:1009B000052F00F2DA81DFE807F0030A0D10133685
:1009C00005230593042105A800F0DEFE17E0544836
:1009D0000421F9E758480421F6E758480421F3E7D1
:1009E0004FF01C08404600F001FF08F10408059094
:1009F000042105A800F0C8FEB8F12C0FF2D10120A7
:100A000000FA07F747EA0B0B5FFA8BFB4FF0000980
:100A100000F0D2FF26B10BF00B030B2B08BF002414
:100A2000FFF76CFE57E746480421CDE7002EA5D01E
:100A30000BF00B030B2BA1D10220FFF757FE07464B
:100A400000289BD0012000F0CFFE0220FFF79EFE81
:100A500000265FFA86F8404600F0D6FE044690B1C4
:100A60000021404600F0E0FE01360028F1D1BA46F0
:100A7000044641F21213022105A8ADF814303E4697
:100A800000F082FE27E70120FFF780FE2546244B79
:100A90009B68AB4207D9284600F0A8FE013040F021
:100AA00067810435F3E7234B00251D70204BBA46C0
:100AB0005D603E46ACE7002E3FF460AF0BF00B03E9
:100AC0000B2B7FF45BAF0220FFF760FE322000F0BB
:100AD0003DFEB0F10008FFF651AF18F003077FF4B8
:100AE0004DAF0F4A926808EB050393423FF646AFBD
:100AF000B8F5807F3FF742AF124B0193B84523DD35
:100B00004FF47A7000F022FE0390039A002AFFF659
:100B100035AF019B039A03F8012B0137EDE700BFC6
:100B200000230020AC24002090230020150700089B
:100B3000B0240020A8230020042300200823002044
:100B40000C230020AC230020C820FFF7CFFD074670
:100B500000283FF413AF1F2D11D8C5F120024245E4
:100B60000AAB25F0030028BF42468349019218448E
:100B700000F0C4FE019A8048FF2100F0D1FE4FEA48
:100B8000A8037D490193C8F38702284600F0D0FEF0
:100B9000064600283FF46DAF019B05EB830537E760
:100BA0000220FFF7A3FD00283FF4E8AE00F04EFE60
:100BB00000283FF4E3AE0027B846704B9B68BB4269
:100BC00018D91F2F11D80A9B01330ED027F0030329
:100BD00012AA134453F8203C05934046042205A969
:100BE00001F014F804378046E7E7384600F0FEFDD0
:100BF0000590F2E7CDF81480042105A800F0C4FDAB
:100C000006E70023642104A8049300F0B3FD002844
:100C10007FF4B4AE0220FFF769FD00283FF4AEAECA
:100C2000049800F009FE0590E6E70023642104A87B
:100C3000049300F09FFD00287FF4A0AE0220FFF790
:100C400055FD00283FF49AAE049800F0F7FDEAE75E
:100C50000220FFF74BFD00283FF490AE00F006FEA7
:100C6000E1E70220FFF742FD00283FF487AE05A927
:100C7000142000F001FE04210746049004A800F0AF
:100C800083FD3946B9E7322000F060FD071EFFF60C
:100C900075AEBB077FF472AE384A926807EB090362
:100CA00093423FF66BAE0220FFF720FD00283FF491
:100CB00065AE27F003074F44B9453FF4A9AE484657
:100CC00000F094FD0421059005A800F05DFD09F1F8
:100CD0000409F1E74FF47A70FFF708FD00283FF4AC
:100CE0004DAE00F0B3FD002844D00A9B01330BD079
:100CF00008220AA9002000F01BFE00283AD020227A
:100D0000FF210AA800F00CFEFFF7F8FC1C4803F0D6
:100D100075FC13B0BDE8F08F002E3FF42FAE0BF042
:100D20000B030B2B7FF42AAE0023642105A8059347
:100D300000F020FD074600287FF420AE0220FFF7D8
:100D4000D5FC804600283FF419AEFFF7D7FC41F2EE
:100D5000883003F053FC059800F044FE464600F04E
:100D60002BFE3C46B7E5064652E64FF0000905E685
:100D7000BA467EE637467CE6AC23002000230020FE
:100D8000A0860100094A136849F2690099B21B0C58
:100D900000FB01331360064B186844F2506182B2C5
:100DA000000C01FB0200186080B270471423002081
:100DB0001023002010B500211022044600F0B0FDE1
:100DC000034B03CB206061601868A06010BD00BFBA
:100DD0009075FF1F2DE9F041ADF54E7D0DF1340802
:100DE0006CAC40F2751207460D460EA80021C8F8FB
:100DF000001000F095FD4FF4C4720021204600F071
:100E00008FFD01F0AFFF274B4FF47A72B0FBF2F089
:100E1000186093E80700012384E807000DF5E970E6
:100E20002382FFF7C7FF41F604531F49238406A816
:100E300004F0A6FA1B2384F832310DF2E32206AB4C
:100E40000DF1300C1E4603CE6645106051603346EE
:100E500002F10802F6D13188B378937011802046F0
:100E60004146012200F0D8FD00230393AB7E02939C
:100E700005F11903019380B20123CDE904800093A9
:100E8000E97E06A3D3E90023384602F02BFB0DF5DB
:100E90004E7DBDE8F08100BFAFF300809E6AC421A3
:100EA000818A46EEB8240020905300082DE9F043D3
:100EB000224DBBB001F056FFAB6840F2ED22C31AE1
:100EC000934232D906AFA8602B462822002138462B
:100ED00002F0B8FC05F10E0000F01AFD00260446F1
:100EE0005FFA80F905F10E08F3B2F100994501F1BE
:100EF000280107D908EB06030822384602F0A2FCB5
:100F00000136F1E708230122CDE9023205340C4B0A
:100F10000193A4B230230093CDE9047405A3D3E96F
:100F20000023297B074802F0DDFA3BB0BDE8F083DF
:100F3000AFF3008078F6339F93CACD8D605E0020BA
:100F40006D5E0020D0340020F0B58B8A013B9BB24F
:100F5000C92BC9B006460C4647D8274D2F7B27BB67
:100F600005F10C03009308223B463946204602F067
:100F70002DFB7B1CFAB2D9001F46A38A013B9A4283
:100F800005DA0E322A44009200230822EEE70023FD
:100F90000022C5E900230023AB6085F8D730C5F8EF
:100FA000D8302B7B0BB9E37E2B738122002106AD59
:100FB00027A800F0B5FC0122294627A800F0FAFD79
:100FC00000230393A37E029304F1190380B20193DB
:100FD0002823CDE90450E17E0093304604A3D3E9F1
:100FE000002302F07FFAFFF761FF49B0F0BD00BFB8
:100FF00026417272DF25D7B7605E002070B50D46BE
:1010000014461E4602F0CAF950B9022E10D1012C26
:101010000ED112A3D3E90023C5E90023012007E084
:10102000282C10D005D8012C09D0052C0FD0002079
:1010300070BD302CFBD10BA3D3E90023ECE70BA34D
:10104000D3E90023E8E70BA3D3E90023E4E70BA3EC
:10105000D3E90023E0E700BFAFF30080401DA120EB
:1010600026812A0B78F6339F93CACD8D9E6AC421C0
:10107000818A46EE26417272DF25D7B7F017304AD3
:1010800039059E562DE9F04F8DB002AF80460D46D2
:1010900002F084F9044600285CD12B7E022B1BD180
:1010A000EB8A012B18D101F05DFE0646FFF76AFEC0
:1010B00003464FF4C870DFF81C92B3FBF0F206F55C
:1010C000167602FB103316FA83F3C9F80030EB7E74
:1010D00033B97B4B00221A702C37BD46BDE8F08F28
:1010E000AB8AE6B2013BB34204F101040CD907F12B
:1010F00008031E44E10000960023082201F0F801D5
:10110000284602F063FAEBE707F11800FFF752FEFA
:10111000324607F1180107F1080004F0FFF8002833
:10112000D7D10F2E08D8664B1E70D9F80030A3F522
:101130001673C9F80030CFE7FB1DF8710146009324
:1011400007220346284602F041FAF979404602F0A8
:101150001DF9C1E7EB8A282B26D010D8012B1ED011
:10116000052BB9D1BFF34F8F5649574BCA6802F4CC
:10117000E0621343CB60BFF34F8F00BFFDE7302B1E
:10118000AAD16B7E514C0133627BDBB29342E946BC
:1011900003D1EA7E237B9A420BD0CD469CE72946B9
:1011A0004046FFF717FE97E729464046FFF7CCFE7B
:1011B00092E74FF0000807F11803A7F818801022F3
:1011C000009341460123284602F000FAAE8A023E0F
:1011D000B6B2F31C9B109B000733DB08A9EBC303DB
:1011E0009D460DF1080A1FFA88F34FEAC8019E4296
:1011F00001F110010AD90AEB080300930822002329
:10120000284602F0E3F908F10108ECE794F8D7006A
:1012100000F0FAFAD4F8D810054619B994F8D700B6
:1012200000F002FBD4F8D83033449D4205D294F844
:10123000D7000021013000F0F7FA4FEA960B4FF08B
:1012400000081FFA88F18B45D4E9003209D90AEB6E
:10125000880103EB8800012200F06AFB08F1010815
:10126000EFE7F31842F10002C4E90032D4F8D830B5
:1012700094F8D70006EB0308C4F8D88000F0C4FA4D
:10128000804509D394F8D730D4F8D8000133401BF7
:1012900084F8D730C4F8D800FF2E0D4D09D80023AC
:1012A000237300F0D3FA00F0C7FC288108B9FFF7D8
:1012B00083FA23689B0A01332B810023A3606CE728
:1012C000C934002000ED00E00400FA05605E002053
:1012D000B8240020CC340020F8B50E4C0E4F022666
:1012E000A4F5805343F8307C237E3BB965692DB16A
:1012F000284600F01FFD284603F0F8FF204600F0C6
:1013000019FDA4F5A554012EA4F1100400D1F8BDD7
:101310000126E5E7E0590020F8530008014B18705A
:10132000704700BFC424002010B54FF000540C4B90
:1013300022689A4211D10B4B627D1A700A48237DB4
:1013400003730A49C9220E3000F0D8FAE0220021C6
:10135000204600F0E5FA012010BD0020FCE700BFA8
:101360009AAD44C5C4240020605E00201600002011
:1013700037B500F061FC1F4C1F4D20492881022326
:101380006B712368204604F580545B6801229847FE
:10139000D4F8B03419495B68012204F59660984787
:1013A00000230193164B174900931748174B4FF42E
:1013B000805201F0C3FF164B197811B1124801F0A9
:1013C000E5FF01F0CFFC0446FFF7DCFC4FF4C873E7
:1013D000B0FBF3F202FB130304F5167010FA83F06E
:1013E0000C4B186003F07EFC08B10F232B8103B077
:1013F00030BD00BF00350020B824002040420F005F
:10140000FD0F0008C8240020D034002085100008FB
:10141000C4240020CC3400202DE9F04F2DED028BA8
:101420009F4D93B0DFF8A0A29E4F284602F086F8A9
:10143000034600283ED00024CDE90F440E94ADF8B9
:101440004440027B8DF8442099684068964E0FAA6C
:1014500003C21B6843F000430E93A046A1463368C5
:10146000D3F810B001F080FC10EB0A0241F1000348
:101470003046CDF800900EA9D84704F22C5440F61F
:1014800058230028C8BF48F0010806F5A5569C421D
:1014900006F11006E3D1B8F1000F05D0284602F09E
:1014A00051F887F80090C0E73B78072B00F2E68000
:1014B00001333B700DF12C089FED738B0023DFF897
:1014C0000C920A93ADF834300B93C8F80430002620
:1014D000754C374601238DF81C3023688DED008B49
:1014E0004FF0000BD3F808A08DF81DB05B460DF14E
:1014F0001D0207A92046D0479DF81CA0BAF1000F95
:1015000024D0D9F8143083F48063C9F81430102241
:1015100059460EA800F004FA236808AA5F690AA9D0
:101520000DF11E032046B84798E803000FAB83E88F
:1015300003009DF834308DF844300A9B0E930EA9B9
:10154000DDE90823284602F0C5F9574606F22C5675
:1015500040F6582304F5A5549E4204F11004B9D175
:10156000002FB4D1284601F019FF002840D14F4E7A
:1015700001F0F8FB336898423AD301F0F3FB0446DC
:10158000FFF700FC4FF4C87304F51674B0FBF3F2D8
:1015900002FB130314FA83F33360454E8DF8287071
:1015A000377817B901238DF82830C7F11004E4B259
:1015B0000EA8FFF7FFFB062C28BF06240EAB224621
:1015C000D9190DF1290000F099F90AAB03931823FA
:1015D00002930134374B0193E4B201230093049446
:1015E0002BA3D3E90023284601F01EFF002333700C
:1015F00001F0B8FB304A314C1368C31AB3F57A7F57
:101600002FD3106001F0B0FB02460B46284601F0D4
:10161000A3FF284601F0C2FE18B3237B284E002BFF
:1016200014BF03230223737101F09CFB0EAF4FF430
:101630007A730122B0FBF3F039463060304600F097
:1016400091FA182302931F4B019380B240F2551375
:10165000CDE90370009328460FA3D3E9002301F0DE
:10166000E3FE237B2BB1FFF721FC237B002B7FF4D0
:10167000D9AE13B0BDEC028BBDE8F08F284601F067
:1016800061FF17E7AFF300800000000000000000DA
:10169000401DA12026812A0BF1C6A7C1D068080FE2
:1016A000D0340020455F002000350020CC340020DD
:1016B000C9340020C8340020405F0020605E002054
:1016C000B8240020445F002040420F00000800487A
:1016D00008B5064800F064FE054800F061FEBDE86C
:1016E0000840044A0449002003F0FABD00350020F8
:1016F000B04900209C5F0020D912000870B5104B43
:101700001B780133DBB2012B0C4612D80D4B1D6840
:1017100029684FF47A730E6AA2FB0332014622460F
:101720002846B047844204D1074B00221A7001209A
:1017300070BD4FF4FA7002F061FF0020F8E700BFBF
:10174000182300201C2300208C5F002007B50023F5
:10175000024601210DF107008DF80730FFF7CEFF9B
:1017600020B19DF8070003B05DF804FB4FF0FF3097
:10177000F9E700000A4608B50421FFF7BFFF80F033
:101780000100C0B2404208BD30B4074B0A46197888
:10179000064B53F821402368DD69054B0146AC46F2
:1017A000204630BC604700BF8C5F00201C23002017
:1017B000A086010070B503F0C9F8094E094D3080CC
:1017C000002428683388834208D903F0BBF82B68CB
:1017D00004440133B4F5104F2B60F2D370BD00BF49
:1017E0008E5F0020485F002003F076B900F10060B2
:1017F00000F510400068704700F10060920000F5AD
:10180000104003F0E9B80000054B1A68054B1B882F
:101810009B1A834202D9104403F094B80020704709
:10182000485F00208E5F0020024B1B68184403F0C5
:10183000A3B800BF485F00200020704700F10050AF
:10184000A0F51040D0F8900570470000064991F8C7
:10185000243033B10023086A81F824300822FFF7CE
:10186000CBBF0120704700BF4C5F0020014B1868C0
:10187000704700BF002004E030B50F4B0F4C1B68D1
:101880002288C3F30B030138934208440BD16468E8
:101890000A46013C824213460BD214F9015F2DB176
:1018A00002F8015BF6E781420B4602D22C2203F8D4
:1018B000012B581A30BD00BF002004E02023002077
:1018C000022802BF024B4FF080629A61704700BF4E
:1018D00000080048022802BF024B4FF480629A6160
:1018E000704700BF00080048022801BF024A536940
:1018F00083F48063536170470008004810B50023EB
:10190000934203D0CC5CC4540133F9E710BD00000E
:1019100003460246D01A12F9011B0029FAD170477A
:1019200002440346934202D003F8011BFAE77047D2
:101930002DE9F8431F4D144695F8242007468846A4
:1019400052BBDFF870909CB395F824302BB920225D
:10195000FF2148462F62FFF7E3FF95F82400C0F10E
:101960000802A24228BF2246D6B24146920005EBA9
:101970008000FFF7C3FF95F82430A41B1E44F6B285
:10198000082E17449044E4B285F82460DBD1FFF7B9
:101990005DFF0028D7D108E02B6A03EB8203834266
:1019A000CFD0FFF753FF0028CBD10020BDE8F8834C
:1019B0000120FBE74C5F0020024B1A78024B1A70A3
:1019C000704700BF8C5F00201823002003494FF4AC
:1019D00061430B60024B186802F0D6BC745F0020B4
:1019E0001C230020094B10B518220446002118467C
:1019F000FFF796FF064A074B127804600146BDE8E0
:101A0000104053F8220002F0BFBC00BF745F0020FA
:101A10008C5F00201C2300202DE9F0470D46044672
:101A200000219046284640F27912FFF779FF2346BD
:101A300020220021284601F005FF231D022220213B
:101A4000284601F0FFFE631D03222221284601F0F3
:101A5000F9FEA31D03222521284601F0F3FE04F11F
:101A6000080310222821284601F0ECFE04F110039F
:101A700008223821284601F0E5FE04F1110308226E
:101A80004021284601F0DEFE04F11203082248211D
:101A9000284601F0D7FE04F11403202250212846E5
:101AA00001F0D0FE04F1180340227021284601F015
:101AB000C9FE04F120030822B021284601F0C2FE2D
:101AC00004F121030822B821284601F0BBFE04F1ED
:101AD0002207C0263B46314608222846083601F038
:101AE000B1FEB6F5A07F07F10107F3D104F132038F
:101AF00008223146284601F0A5FE002704F1330AEA
:101B000094F832304FEAC7099F4209F5A47615D3FD
:101B1000B8F1000F08D1314604F599730722284621
:101B200001F090FE09F24F16274694F832213B1B34
:101B300093420CD3F01DC008BDE8F0870AEB070301
:101B400008223146284601F07DFE0137D8E707F22A
:101B5000331331460822284601F074FE0836013757
:101B6000E3E7000013B50446084600210160234660
:101B7000C0F803102022019001F064FE0198231D9B
:101B80000222202101F05EFE0198631D0322222122
:101B900001F058FE0198A31D0322252101F052FEF9
:101BA000019804F108031022282101F04BFE0720C0
:101BB00002B010BDF8B50E4605461446002181223C
:101BC0003046FFF7ADFE2B4608220021304601F0DB
:101BD00039FE7CB96B1C07220821304601F032FE29
:101BE0000F2401236A785F1C013B934204D3E01D5C
:101BF000C008F8BD0824F4E7EB1921460822304656
:101C000001F020FE08343B46ECE7000030B5094DFA
:101C10000A4491420DD011F8013B5840082340F38B
:101C20000004013B2C4013F0FF0384EA5000F6D17E
:101C3000EFE730BD2083B8ED73B5384A10685168BE
:101C40006B4603C36A4636493648082303F076FBE1
:101C5000044670B9344A106851686B4603C36A463B
:101C600032493048082303F069FB044630BB0A20A0
:101C700022E00369B3F5EE2FECD8418B40F21D4210
:101C80009142E7D12A4A024402F110018B42E1D38A
:101C9000103B244900209D1AFFF7B8FF2A4606464C
:101CA00004F118010020FFF7B1FFA3689E42D1D1D3
:101CB000E3689842CED1002002B070BD0369B3F54D
:101CC000EE2F22D8B0F8661040F21D4291421ED18C
:101CD000174A024402F15C018B421AD35C3B114962
:101CE00000209D1AFFF792FF2A46064604F1640180
:101CF0000020FFF78BFFA268964203460BD1E068F5
:101D0000834214BF0D200020D6E70B20D4E70C201F
:101D1000D2E71020D0E70D20CEE700BFB85300086F
:101D2000DC6F070000900008C1530008906F0700A7
:101D30000870FFF710B5037C044613B9006803F080
:101D4000E5FA204610BD00000023BFF35B8FC3609F
:101D5000BFF35B8FBFF35B8F8360BFF35B8F704715
:101D6000BFF35B8F0068BFF35B8F704770B50546AC
:101D70000C30FFF7F5FF05F1080604463046FFF783
:101D8000EFFFA04206D930466D68FFF7E9FF254412
:101D9000281A70BD3046FFF7E3FF201AF9E700006C
:101DA00070B50546406898B105F10800FFF7D8FF07
:101DB00005F10C0604463046FFF7D2FF8442304658
:101DC00094BF6D680025FFF7CBFF013C2C44201A1F
:101DD00070BD000038B50C460546FFF7C7FFA042AE
:101DE00010D305F10800FFF7BBFF04446868B4FB9B
:101DF000F0F100FB1144BFF35B8F0120AC60BFF337
:101E00005B8F38BD0020FCE72DE9F0411446074602
:101E10000D46FFF7C5FF844228BF0446D4B1B8463B
:101E200058F80C6B4046FFF79BFF30442860404653
:101E30007E68FFF795FF331A9C4203D86C6001203F
:101E4000BDE8F0816B60A41B3B68AB602044E86098
:101E50000220F5E72046F3E738B50C460546FFF7C4
:101E60009FFFA04210D305F10C00FFF779FF044457
:101E70006868B4FBF0F100FB1144BFF35B8F0120F5
:101E8000EC60BFF35B8F38BD0020FCE72DE9FF411C
:101E9000884669460746FFF7B7FF6C4606B204EB73
:101EA000C6060025B44209D06268206808EB050127
:101EB000FFF724FD636808341D44F3E729463846DC
:101EC000FFF7CAFF284604B0BDE8F081F8B5054623
:101ED0000C300F46FFF744FF05F108060446304674
:101EE000FFF73EFFA042304688BF6C68FFF738FF1F
:101EF000201A386020B130462C68FFF731FF2044AB
:101F0000F8BD000073B5144606460D46FFF72EFFD8
:101F1000844228BF04460190DCB101A93046FFF796
:101F2000D5FF019B33B93268C5E90233C5E9002406
:101F300001200CE09C4238BF019428600198686041
:101F40008442F5D93368AB60241AEC60022002B0F9
:101F500070BD2046FBE700002DE9FF410F466946B2
:101F6000FFF7D0FF6C4600B204EBC0050026AC4280
:101F700009D0D4F8048054F8081BB8194246FFF77A
:101F8000BDFC4644F3E7304604B0BDE8F0810000F4
:101F900038B50546FFF7E0FF044601462846FFF73F
:101FA00019FF204638BD0000302383F3118862B644
:101FB00070470000002383F3118862B67047000069
:101FC000012070477047000010B41346026814687F
:101FD0000022A4465DF8044B6047000000F58050E5
:101FE00090F859047047000000F5805090F85204B2
:101FF0007047000000F5805090F9580470470000C9
:102000005020704700F5805208B5FFF7CDFFD2F899
:102010009834D2F894041844D2F890341844D2F882
:1020200078341844D2F888341844D2F884341844E8
:10203000FFF7C0FF08BD000038B5C26A936923F0FE
:1020400001039361044600F08DFE0546E36A9B6937
:10205000DB0706D500F086FE431BFA2BF6D90020DD
:1020600004E004F58054012084F8520438BD0000D7
:102070002DE9F04F0C4600F5805185B01F4691F8D0
:102080005234BDF83890054690469BB1D1F874346F
:102090000133C1F8743423689A0006D4237B082BDB
:1020A0000BD9627B0AB10F2B07D9D1F878340133F1
:1020B000C1F878344FF0FF300FE0FFF775FFEB6A9F
:1020C000D3F8C42012F4001A0AD0D1F87C340133BA
:1020D000C1F87C34FFF76EFF002005B0BDE8F08F3B
:1020E000D3F8C46022686B6AC6F301464FF0480B10
:1020F000002A1BFB063BB4BF42F080429204CBF89F
:10210000002023685B0044BF42F00052CBF800205F
:10211000227B330643EA0243CBF80430607B720132
:1021200018B343F44013CBF80430D1F8A43401338E
:10213000C1F8A434AB1803F58353197B41F0200197
:102140001973207B039200F06BFE039A033080101A
:102150005FFA8AF383420AF1010A0DDA04EB830184
:102160000BEB830349689960F2E7AB1803F58353DF
:10217000197B60F34511E3E7EB6A0121B140C3F835
:10218000CC10AB1803F58253C3E9048705EB461363
:1021900003F582532146183304F10C0051F804CBA7
:1021A00043F804CB8142F9D1098819802A4441F2CD
:1021B00068032846D65002F5805209F0030392F8CE
:1021C0006C1043F0100321F01F010B4382F86C30B8
:1021D000FFF7F0FE4246CDF800903B46214600F066
:1021E000E5FD012079E7000013B500F58054019169
:1021F000606CFFF7D5FD1F280AD90199606C202279
:10220000FFF744FEA0F120035842584102B010BD30
:102210000020FBE708B500F58050FFF7C5FE406CD5
:10222000FFF792FDBDE80840FFF7C4BE0022026040
:10223000828142608260704710B500220023C0E9AD
:1022400000230023044603810C30FFF7EFFF2046F4
:1022500010BD00002DE9F047074688B007F580540F
:1022600068469A468846FFF79FFE9146FFF7E4FFCF
:10227000606CFFF77BFD1F282CD9606C202269461B
:10228000FFF786FE202825D194F8523413B303AD0E
:10229000444605AB2E4603CE9E4220606160354623
:1022A00004F10804F6D130682060B388A380DDE92A
:1022B0000023C9E90023BDF80830AAF80030FFF771
:1022C00079FE4A4653464146384608B0BDE8F047D5
:1022D00000F05ABDFFF76EFE002008B0BDE8F087A1
:1022E0002DE9F84F00230646C0E90133294B46F893
:1022F000303B00F581540546884637461034384651
:102300002037FFF799FFA742F9D105F580544FF424
:10231000805326630026C4E90D366764012305F562
:10232000835705F5A359E66384F8403084F84830B4
:10233000103709F110094FF0000A4FF0000B47E980
:1023400008ABA7F11800FFF771FF203747F8286C9A
:102350004F45F4D1B8F1010F84F85884A4F85A64B9
:10236000A4F85C64A4F85E6484F86064A4F8626411
:10237000A4F86464A4F8666484F8686402D9064822
:1023800000F0EAFC054B53F82830EB622846BDE824
:10239000F88F00BFF8530008CC530008E85300083A
:1023A00010B5044B197804464A1C1A70FFF798FFC1
:1023B000204610BD995F00202DE9F04300295FD031
:1023C0003048314BB3FBF1F381428CBF0A2011201E
:1023D000451EB3FBF0F700FB1730ECB220B1022D25
:1023E0002846F5D8002037E07D1EB5F5806F33D242
:1023F000C4EBC40808F103034FEAE30EC3F3C703B9
:10240000A4EB030C0EF101094FF47A705FFA8CF61D
:102410000EFB000E59FA8CFCBEFBFCFCBCF5617F88
:102420001CDC1FFA8CF4581C56FA80F047431648FF
:10243000B0FBF7F7B942D5D1013BDBB20F2BD1D8B6
:10244000711EC9B207294FF0000005D81071148021
:102450005580537191710120BDE8F08308F1FF337D
:102460004FEAE30CC3F3C703E41A0CF1010EE6B222
:102470000CFB00005EFA84F4B0FBF4F4A4B2D2E7E3
:102480000846E9E73F420F000024F40038B500F5A4
:102490008053114A93F85834D55C4FF45472554325
:1024A00005F1804303F52443044600211846FFF755
:1024B00037FA0A4B60612B44A361094B2B44E3615B
:1024C000084B2B442362084B2B446362E36A0022CF
:1024D000C3F8C02038BD00BFE053000870A400401E
:1024E000B0A4004088A5004078A600402DE9F04F38
:1024F00000F58055994695F85834022B89B004466A
:102500008A46904604D90027384609B0BDE8F08FC6
:102510009C4A52F8231009B942F823009A49C4F89A
:102520000CA00B7884F8109093B9FFF73DFD974B02
:102530009A6D42F000729A659A6B42F000729A634B
:102540009A6B22F000729A6301230B70FFF732FD41
:1025500095F85134BBB9FFF727FD8D4A95F85834EB
:10256000D35C012B26D0022B2BD03BB903211520A5
:1025700001F054FD0321162001F050FD012385F8E0
:102580005134FFF717FDFFF70FFDE26A936923F05F
:102590001003936100F0E6FB0746E36A9E6916F0BC
:1025A000080615D000F0DEFBC31BFA2BF5D9FFF7A8
:1025B00001FDA8E70321562001F030FD032157203B
:1025C000DAE70321582001F029FD03215920D3E740
:1025D0009A6942F001029A6100F0C4FB0746E36A7F
:1025E0009A69D00705D400F0BDFBC31BFA2BF6D9BE
:1025F000DDE79A6942F002029A61E36A00275F65AB
:10260000FFF7D8FC686CFFF79FFB04F5825B0BF1CA
:10261000100B202200216846FFF782F902A8FFF77D
:1026200005FE06976A460BEB06030DF1180E94465D
:10263000BCE80300F44518605960624603F10803E2
:10264000F5D1DCF80000186020369CF804201A71DF
:10265000B6F5806FDDD1002304F5A25285F8503421
:1026600085F853341A3251462046FFF7A5FE074637
:1026700090B9E26A936923F00103936100F072FB61
:102680000546E36A9B69D9077FF53DAF00F06AFB19
:10269000431BFA2BF5D936E795F85F6495F85E246D
:1026A000C5F86CA4360246EA426695F86024E36AEF
:1026B0001643B5F85C2446EA0246DE61B8F1000F25
:1026C00029D004F5A352023241462046FFF774FE9A
:1026D00090B9E26A936923F00103936100F042FB31
:1026E0000546E36A9B69DA077FF50DAF00F03AFB18
:1026F000431BFA2BF5D906E795F8683495F867146B
:10270000C5F870841B0143EA0123B5F86414E26A3A
:1027100043EA0143D3602046FFF7B8FE002385F863
:102720005934E36A6FF040421A65E36A194A5A6500
:10273000E36A44229A65E36A0722C3F8DC20E36A6D
:102740000322DA65E26A9369B9F1030F43F4407337
:1027500093613FF4D9AEE26A936923F00103936178
:1027600000F000FB0646E36A9B69DB0705D500F035
:10277000F9FA831BFA2BF6D9C5E6012385F8523402
:10278000C2E600BF905F0020985F0020001002406A
:10279000E05300089B0008002DE9F04F054689B082
:1027A00090469946002741F2680A00F58056EB6A88
:1027B000D3F8D430FB40D8074AD505EB4712524432
:1027C0004FEA471B1379190742D4D6F880340133F6
:1027D000C6F8803413799A0648BFD6F8A83405EBBA
:1027E0000B0248BF0133524448BFC6F8A8341379DE
:1027F00043F008031371DB0722D596F85334FBB17D
:1028000005F58254183468465C44FFF715FD03ABA8
:1028100004F1080C206861681A4603C20834644554
:102820001346F7D120681060A2889A800123ADF882
:1028300008302B68CDE90089DB6B6946284698474C
:10284000D6F8543423B1D6F89C340133C6F89C34FE
:102850000137202FABD109B0BDE8F08F2DE9F04F43
:102860008DB004460F4600F07FFA82468946002F5D
:1028700056D1E36AD3F89020920141BF04F580510C
:10288000D1F894240132C1F89424D3F8902016078B
:1028900003D100200DB0BDE8F08FD3F89050E66969
:1028A000C5F30125482303FB0566E8464046FFF7CC
:1028B000BDFC326851004ABF22F06043C2F38A4334
:1028C00043F00043920048BF43F080430093736895
:1028D00013F400131FBF04F5805201238DF80D304F
:1028E000D2F8AC340EBF8DF80D300133C2F8AC34E1
:1028F000F38803F00F038DF80C304FF0000B9DF8B8
:102900000C0000F08DFA5FFA8BF3984220D9F21890
:102910000CA90B44127A03F82C2C0BF1010BEEE7F7
:10292000012FB6D1E36AD3F89820950141BF04F591
:102930008051D1F894240132C1F89424D3F898201E
:102940001007A6D0D3F89850266AC5F30125A9E749
:10295000EFB9E36AC3F8945004A8FFF76DFC98E858
:102960000F0007AD07C52B800023ADF81830236892
:102970002046CDE904A9DB6B04A9984704F58054EF
:1029800058B1D4F88C340133C4F88C3482E7012F69
:1029900004BFE36AC3F89C50DEE7D4F890340133F7
:1029A000C4F89034012075E7F8B505460F4600F5E8
:1029B0008054012639462846FFF750FF10B184F8AD
:1029C0005364F7E7D4F8543423B1D4F89C3401337A
:1029D000C4F89C34F8BD0000F0B5C36A1A6C12F458
:1029E0007F0F2BD000F580541B6CC4F8A03441F24B
:1029F0006805002347194FF0010C00EB43122A44ED
:102A00005E01117911F0020F15D0490713D4B9599D
:102A1000C66AD6F8C8E00CFA01F111EA0E0F0AD026
:102A2000C6F8D010117941F004011171D4F888244E
:102A30000132C4F888240133202BDED1F0BD000020
:102A40002B4B70B51E561B5C012B2FD8294D2A4AE3
:102A500055F8233052F826400BB341B3236D1A06C4
:102A60000FD58023236500F07FF950EA01020B4661
:102A700002D0013861F10003024655F82600FFF745
:102A80008BFE236D1B032CD555F826304FF4002206
:102A900003F580532265012283F8592421E00123A4
:102AA0002365082323654FF48063236570BD236D80
:102AB000DA0702D4236D9B0706D5032355F82600B9
:102AC00023650021FFF770FF236D180702D4236DE3
:102AD000D90606D5182355F8260023650121FFF7EE
:102AE00063FF55F82600BDE87040FFF775BF00BFD3
:102AF000E4530008905F0020E853000808B5FFF792
:102B000053FAFFF769FFBDE80840FFF753BA00002A
:102B1000C36AD3F8C40080F40010C0F3405070477B
:102B200000F5805008B5FFF73FFA406CFFF71EF93B
:102B3000FFF740FA43090CBF0120002008BD000048
:102B400000F5805393F8592462B1C16A8A6922F072
:102B500001028A61D3F898240132C3F89824002234
:102B600083F85924704700002DE9F74300F582519E
:102B700098461031FFF718FA002541F2680E4FF021
:102B8000010900F5805C00EB4514744423795E076D
:102B90001CD4DB061AD5C36A8E69D3F8C87009FA4B
:102BA00006F63E4212D04F6801970F689742019F88
:102BB00077EB08070AD2C3F8D060237943F0040307
:102BC0002371DCF884340133CCF884340135202DB2
:102BD00001F12001D7D103B0BDE8F043FFF7EAB916
:102BE000F8B51E46002313700F4605461446FFF73E
:102BF00097FF80F0010038701EB12846FFF788FF6C
:102C00002070F8BD2DE9F04F85B09946DDE90EA39F
:102C10000D4602931378019391F800B08046164652
:102C200000F0A2F82B7804460F4613B93378002B36
:102C300042D022463B464046FFF796FFFFF75EFF35
:102C4000FFF77EFF4B4632462946FFF7C9FF2B7838
:102C500033B1BBF1000F03D0012005B0BDE8F08F08
:102C6000337813B1019B002BF6D108F58053039301
:102C7000029B544577EB03031ED2039BD3F8540405
:102C8000D0B10368AAEB0401DB6889B298474B46D0
:102C9000324629464046FFF7A3FF2B7813B1BBF11C
:102CA000000FD9D1337813B1019B002BD4D100F0A0
:102CB0005BF804460F46DBE70020CEE708B50021AD
:102CC0000846FFF7BDFEBDE8084001F05FB8000010
:102CD00008B501210020FFF7B3FEBDE8084001F070
:102CE00055B8000008B500210120FFF7A9FEBDE896
:102CF000084001F04BB8000008B501210846FFF775
:102D00009FFEBDE8084001F041B8000000B59BB04F
:102D1000EFF3098168226846FEF7F0FDEFF30583C3
:102D2000014B9B6BFEE700BF00ED00E008B5FFF72D
:102D3000EDFF000000B59BB0EFF309816822684603
:102D4000FEF7DCFDEFF30583014B5B6BFEE700BF95
:102D500000ED00E0FEE700000FB408B5029801F0B6
:102D6000E3FBFEE701F006BF01F0DEBE01F0DCBED2
:102D700013B56C4684E80600031D94E8030083E85D
:102D80000500012002B010BD73B58568019155B1F1
:102D90001B885B0707D4D0E900369B6B9847019AE4
:102DA000C1B23046A847012002B070BDF0B58668B8
:102DB00089B005460C465EB1BDF838305B070AD4D1
:102DC000D0E900379B6B98472246C1B23846B047DE
:102DD000012009B0F0BD00220023CDE9002300232B
:102DE000ADF808300A4603AB01F1080610685168D7
:102DF0001C4603C40832B2422346F7D11068206053
:102E00009288A280FFF7B2FF0423ADF808302B6848
:102E1000CDE90001DB6B694628469847D8E70000FA
:102E2000082817D909280CD00A280CD00B280CD058
:102E30000C280CD00D280CD00E2814BF40203020B8
:102E400070470C20704710207047142070471820DE
:102E500070472020704700002DE9F041456A15B900
:102E60004162BDE8F0814B6823F06047C3F38A46B6
:102E70004FEAD37EC3F3807816EA230638BF3E4676
:102E8000AC462B465A68BEEBD27F22F060440AD093
:102E9000002A18DAA40CB44217D19D420FD10D605C
:102EA000DEE71346EEE7A74207D102F08044C2F303
:102EB000807242450BD054B1EFE708D2EDE7CCF871
:102EC00000100B60CDE7B44201D0B442E5D81A68D7
:102ED0009C46002AE5D11960C3E700002DE9F047C0
:102EE000089D01F007044FEAD508224405F00705C4
:102EF00000EBD1004FF47F49944201D1BDE8F08747
:102F000004F0070705F0070A57453E4638BF564606
:102F1000C6F10806111B8E4228BF0E46E10808EBD9
:102F2000D50E415C13F80EC0B94029FA06F721FA14
:102F30000AF1FFB28CEA010147FA0AF739408CEA3C
:102F4000010C03F80EC034443544D5E780EA012073
:102F5000082341F2210201B24000002980B203F1AE
:102F6000FF33B8BF504013F0FF03F4D170470000A7
:102F700038B50C468D18A54200D138BD14F8011B98
:102F8000FFF7E4FFF7E7000042684AB113684360C7
:102F90004389818901339BB29942438138BF838140
:102FA0001046704770B588B0202204460D4668462A
:102FB0000021FEF7B5FC20460495FFF7E5FF024629
:102FC00058B16B46054608AE1C4603CCB442286097
:102FD0006960234605F10805F6D1104608B070BDBA
:102FE000082817D909280CD00A280CD00B280CD097
:102FF0000C280CD00D280CD00E2814BF40203020F7
:1030000070470C207047102070471420704718201C
:103010007047202070470000082817D90C280CD9C9
:1030200010280CD914280CD918280CD920280CD910
:1030300030288CBF0F200E207047092070470A20CF
:1030400070470B2070470C2070470D207047000020
:103050002DE9F843078C072F04461ED9D0E90298C2
:1030600000254FF6FF73C5F12006A5F1200029FACF
:1030700005F108FA06F628FA00F031430143C9B217
:103080001846FFF763FF0835402D0346EBD1E16991
:103090003A46BDE8F843FFF76BBF4FF6FF70BDE857
:1030A000F883000010B54B6823B9CA8A63F309029C
:1030B000CA8210BD04691A681C600361C38A013B9F
:1030C000C3824A60EFE700002DE9F84F1D46CB8A26
:1030D0000F46C3F309010529814692460B4630D0BD
:1030E0000020AAB207F11A049EB2042E1FFA80F83B
:1030F0000FD8904503F1010306D3FB8A0A4462F31B
:103100000903FB8201201AE01AF80060E65401303E
:10311000EAE79045F1D2A1F1050B1C237C68BBFBCB
:10312000F3F203FB12BB1FFA8BF6002C45D1484685
:10313000FFF72AFF044638B978606FF00200BDE857
:10314000F88F4FF00008E6E7002606607860ADB221
:103150004FF0000B454510D90AEB0803221D13F868
:10316000011B9155B1B208F101081B291FFA88F81B
:103170002BD0454506F10106F1D8FB8AC3F30902BD
:10318000154465F30903BCE7013292B21C4623687B
:10319000002BF9D16B1F0B441C21B3FBF1F301335E
:1031A0009BB29A42D3D2BBF1000FD0D14846FFF771
:1031B000EBFE20B9C4F800B0BFE70122E7E7C0F892
:1031C00000B05E4620600446C1E74545D5D9484673
:1031D000FFF7DAFE08B92060AFE7C0F800B00026BC
:1031E00020600446B6E700002DE9F04F2DED028B7C
:1031F0001C4683B05B69019207468846002B00F0AD
:103200009A80238C2BB1E269002A00F09480072B6E
:1032100035D807F10C00FFF7B7FE054638B96FF057
:103220000205284603B0BDEC028BBDE8F08F1422E6
:103230000021FEF775FB228CE16905F10800FEF71D
:103240005DFB208C013080B2FFF7E6FEFFF7C8FE81
:10325000013880B22084013028746369228C1B7885
:103260002A4403F01F0363F03F0348F00041137248
:10327000384669602946FFF7EFFD0125D1E700F1E7
:103280000C034FF0000908EE103A4FF0800A4E464A
:103290004D4618EE100AFFF777FE83460028BED091
:1032A00014220021FEF73CFB002E3AD1019BABF823
:1032B000083002220BF1080E1FFA82FC0CF101000B
:1032C000BCF1060F218C80B201D88E422BD3FFF7C0
:1032D000A3FEFFF785FE62691278013802F01F0233
:1032E0008E4208BF4FF0400A42EA49121BFA80F1B1
:1032F0004AEA020A013048F0004281F808A08BF83F
:103300001000CBF8042059463846FFF7A5FD238C62
:103310000135B3422DB289F001094FF0000AB8D14E
:103320007FE70022C6E7E169895D0EF802100136E9
:10333000B6B20132C0E76FF0010572E7F8B5154685
:103340000E463022002104461F46FEF7E9FA069B8E
:103350006360B5F5001F079BA76034BF6A094FF68D
:10336000FF72A36297B2E66104F1100000239A4253
:1033700006D800230360A782E3822383E360F8BDBD
:103380000660013330462036F1E7000003781BB9B0
:103390004BB2002BC8BF0170704700000078704727
:1033A000F8B50C46C969074611B9238C002B37D1F3
:1033B000257E1F2D34D8387828BB228C072A2CD89C
:1033C000268A36F003032BD14FF6FF70FFF7D0FDAE
:1033D00020F001003102400441EA0561400C41EA5D
:1033E00040254FF6FF72234629463846FFF7FCFE7C
:1033F000002807DD626913780133DBB21F2B88BF19
:1034000000231370F8BD218A2D0645EA01250543E6
:103410002046FFF71DFE0246E5E76FF00300F1E7E7
:103420006FF00100EEE7000070B58AB00446164662
:103430000021282268461D46FEF772FABDF8383092
:10344000ADF810300F9B05939DF840308DF8183083
:10345000119B07936946BDF84830ADF820302046EF
:10346000CDE90265FFF79CFF0AB070BD2DE9F04180
:10347000D36905460C4616460BB9138C5BBB377EE9
:103480001F2F28D895F80080B8F1000F26D03046BD
:10349000FFF7DEFD3378210241EAC33141EA08013A
:1034A000338A41EA076141EA03410246334641F06B
:1034B00080012846FFF798FE00280ADD3378012BAB
:1034C00007D1726913780133DBB21F2B88BF002349
:1034D0001370BDE8F0816FF00100FAE76FF00300B0
:1034E000F7E70000F0B58BB004460D461746002103
:1034F000282268461E46FEF713FA9DF84C305A1EE5
:10350000534253418DF800309DF84030ADF81030F3
:10351000119B05939DF848308DF81830149B079344
:103520006A46BDF85430ADF8203029462046CDE932
:103530000276FFF79BFF0BB0F0BD0000406A00B1C0
:1035400004307047436A1A68426202691A60036174
:10355000C38A013BC38270472DE9F041D0F8208037
:10356000194E14461D464146002709B9BDE8F081B1
:10357000D1E90223A21A65EB0303964277EB03031A
:103580001ED2036A8B420DD1FFF78CFD036A1B68C4
:10359000036203690B60C38A0161016A013BC38254
:1035A0008846E2E7FFF77EFD0B68C8F80030036944
:1035B0000B60C38A0161013BC382D8F80010D4E7D5
:1035C00088460968D1E700BF80841E002DE9F04FCE
:1035D0008BB00D46DDF8509014469B46804600287F
:1035E00000F01981B9F1000F00F01581531E3F2B37
:1035F00000F21181012A03D1BBF1000F40F00B81D1
:103600000023CDE90833B8F81430B5EBC30F4FEA07
:10361000C30703D300200BB0BDE8F08F2B199F42E6
:10362000D8F80C303ABF7F1BFFB227461BB9D8F839
:103630001030002B7AD0272D4ED8C5F12806B7427E
:103640004FF000032CBFF6B23E4600932946D8F84F
:10365000080008AB3246FFF741FCA7EB060A3544E9
:103660005FFA8AFAB8F8143003F10053053BDB0027
:103670000493D8F80C3003932821039B13B1BAF1BB
:10368000000F2CD1D8F8100040B1BAF1000F05D0CE
:10369000009608AB5246691AFFF720FC38B2002F9B
:1036A000B8D066070AD00AAB03EBD401624211F826
:1036B000083C02F00702134101F8083C082C3CD9F1
:1036C000102C40F2B580202C40F2B780BBF1000FE7
:1036D00000F09C80082334E0BA460026C2E7049B31
:1036E000E02B28BFE02306930B44AB42059314D98B
:1036F0005A1B03980096924534BF5246D2B2691ABB
:1037000008AB04300792FFF7E9FB079A1644AAEBCF
:10371000020A1544F6B25FFA8AFA049B069A0599E2
:103720009B1A0493039B1B680393A6E70093D8F8A6
:10373000080008AB3A462946AEE7BBF1000F13D0AC
:103740000123B4EBC30F6CD0082C12D89DF82030A5
:10375000621E23FA02F2D50706D54FF0FF3202FAB5
:1037600004F423438DF820309DF8203089F8003090
:1037700051E7102C12D8BDF82030621E23FA02F255
:10378000D10706D54FF0FF3202FA04F42343ADF817
:103790002030BDF82030A9F800303CE7202C0FD8AD
:1037A0000899631E21FA03F3DA0705D54FF0FF32BB
:1037B00002FA04F40C430894089BC9F800302AE785
:1037C000402C2BD0DDE90865611EC4F12102A4F173
:1037D000210326FA01F105FA02F225FA03F3114357
:1037E0001943CB0712D50122A4F12003C4F1200113
:1037F00002FA03F322FA01F1A240524243EA010322
:1038000063EB430332432B43CDE90823DDE908236F
:10381000C9E90023FFE66FF00100FCE66FF0080045
:10382000F9E6082CA0D9102CB3D9202CEED8C3E788
:10383000BBF1000FADD0022383E7BBF1000FBBD07B
:1038400004237EE730B5012A144638BF0124402CFA
:1038500085B028BF40240025012ACDE9025518D89B
:103860001B788DF8083063070AD004AB03EBD4054E
:10387000624215F8083C02F00702934005F8083C44
:10388000009103462246002102A8FFF727FB05B05E
:1038900030BD082AE4D9102A03D81B88ADF80830B7
:1038A000E1E7202A8DBFD3E900231B680293CDE90D
:1038B0000223D8E710B5CB681BB98B600B618B82F4
:1038C00010BD04691A681C600361C38A013BC3828E
:1038D000CA60F0E72DE9F04F93B0CDE903230B6800
:1038E00004460D461806C3F3C01147BFC3F3C03BDF
:1038F000C3F306264FF0020B0E46002B80F2FF8129
:1039000013F0C04940F0FB812A7B002A00F0F781C8
:10391000BBF1020F03D02078B04240F0F381C3F333
:103920000460079003F07F00059059B3C3F3074A82
:103930002A44059B92F80380760646EA0B4646EA3F
:10394000834600220023CDE908235FEAD81346EA24
:103950000A0602936AD0059B009367685B4652464D
:1039600008A92046B847002800F0CF81276A87B908
:10397000314604F10C00FFF715FB0746C8B96FF09C
:10398000020057E0C3F30F2A590608BF0AF0030AE2
:10399000CEE73B699E420DD03F68002FF9D13146FA
:1039A00004F10C00FFF7FEFA07460028E7D0236A6F
:1039B0003B602762FE7D08F01F03C6F38406F01A01
:1039C0001FFA80FC0028B8BF0CF12000D7E90221C3
:1039D0000693A3EB06031FFA83FCB8BF00B2002BCB
:1039E000BCBF0CF120031BB252EA010636D0039E85
:1039F000DFF8D4C2B21A049E66EB0101002694459A
:103A000076EB010C2AD395F80DE097F81AC0E6453D
:103A100018D1029E002E79D001281FDC7868E8B901
:103A2000A84E964270EB010216D337E0276A27B9F9
:103A30006FF00C0013B0BDE8F08F3B699E42B9D027
:103A40003F68F4E79F48904276EB010201D30020E3
:103A5000F0E7029A002AFAD00F2B18DCFA7D4FEA21
:103A6000880302F0030203F07C031343FB7539461D
:103A70002046FFF717FB6B7BBB76029B3BB9FB7DB8
:103A8000C3F38402013262F38603FB75D0E76A7BDD
:103A9000BB7E9A42DBD1029B002B37D04FEA9813B2
:103AA000022B33D0039BBB60049BFB6014220021DC
:103AB0000DA8FDF735FF039B0A93049B0B932B1D69
:103AC0000C932B7BADF83EA0013BDBB2ADF83C3054
:103AD000069B8DF84130079B8DF84230059B8DF891
:103AE000433094F82C308DF840B083F001038DF80A
:103AF00044300AA9A36820469847FB7DC3F384039A
:103B0000013303F01F039B02FB82A0E7FB7DC8F398
:103B10004012B2EBD31F40F0FB80069AC3F384033C
:103B2000934240F0F88002992B7B4FEA98120029CB
:103B30004DD0D2075DD4032B40F2F080039BBB60D5
:103B4000049BFB602B7BAE1D033BDBB23246394648
:103B500004F10C00FFF7B8FA00280CDA39462046C9
:103B6000FFF7A0FAFB7DC3F38403013303F01F03C7
:103B70009B02FB8203E7DDE90884AB883B834FF6B9
:103B8000FF73C9F12000A9F1200228FA09F104FA13
:103B900000F0014324FA02F211431846C9B2FFF7BC
:103BA000D5F909F10809B9F1400F0346E9D1B88206
:103BB0002A7B033AD2B23146FFF7DAF9FB7DB882AD
:103BC000DA43C2F3C01262F3C713FB753FE782B951
:103BD0002E1D013BDBB23246394604F10C00FFF7E3
:103BE00073FA0028BADB2A7BB88A013AD2B231468E
:103BF000E2E7F98AC1F30901013B0429DAB25CD892
:103C0000281D002307F11B069A4208D910F801CBA2
:103C100006F801C0013101330529DBB2F4D1039963
:103C20000A9104990B91934207F11B010C9138BF43
:103C3000043379680D9134BF55FA83F300230E9352
:103C4000FB8AADF83EA0C3F309031A44069B8DF826
:103C50004130079B8DF84230059B8DF8433094F836
:103C60002C30ADF83C2083F001038DF84430002364
:103C70008DF840B07B602A7BB88A013A291DFFF796
:103C800077F93B8BB882834203D1A3680AA9204607
:103C9000984720460AA9FFF70DFEFB7DBA8AC3F3B9
:103CA0008403013303F01F039B02FB823B8B9A4288
:103CB0000CBF00206FF01000BCE67B68002BAED07C
:103CC000052005E040420F0080841E001C30334672
:103CD0001E68002EFAD1091A081D2E1D184401EB8A
:103CE000090CBCF11B0F5FFA89F398D89A4296D958
:103CF00016F8013B00F8013B09F10109EFE76FF00D
:103D0000090097E66FF00A0094E66FF00B0091E669
:103D10006FF00D008EE66FF00E008BE66FF00F0077
:103D200088E600BFEFF3098305494A6B22F00102E0
:103D30004A63683383F30988002383F3118870474B
:103D400000EF00E0302080F3118862B60C4B0D4A82
:103D5000D96821F4E0610904090C0A43DA60D3F858
:103D6000FC20094942F08072C3F8FC200A6842F046
:103D700001020A602022DA7783F82200704700BF30
:103D800000ED00E00003FA05001000E010B530235C
:103D900083F311880E4B5B6813F4006314D0F1EECB
:103DA000103AEFF30984683C4FF08073E361094BEC
:103DB000DB6B236684F3098800F074FB10B1064BBB
:103DC000A36110BD054BFBE783F31188F9E700BF42
:103DD00000ED00E000EF00E04306000846060008A2
:103DE000026843681143016003B11847704700003F
:103DF000024A136843F0C003136070470044004058
:103E000013B50E4C204600F0B3FA04F114000C492F
:103E1000009400234FF4807200F070F9094B0A49B6
:103E200000944FF4807204F1380000F0E9F9074A79
:103E3000074BC4E9172302B010BD00BFA05F0020EC
:103E40000C600020F13D00080C610020004400409F
:103E5000007A030A30B5037C214C002918BF0C46B8
:103E6000012B0CD11F4B984209D11F4B9A6D42F484
:103E700000329A659A6F42F400329A679B6F22680B
:103E8000036EC16D846603EB5203B3FBF2F3626809
:103E9000150442BF23F0070503F0070343EA450377
:103EA000CB60A36843F040034B60E36843F0010339
:103EB0008B6042F4967343F001030B604FF0FF33C5
:103EC0000B62510505D512F0102205D0B2F1805FCA
:103ED00004D080F8643030BD7F23FAE73F23F8E751
:103EE00038540008A05F0020001002402DE9F04780
:103EF000C66D3768F46934622107054619D014F09D
:103F0000080118BF4FF48071E20748BF41F020015B
:103F1000A30748BF41F04001600748BF41F080015E
:103F2000302383F31188281DFFF75AFF002383F302
:103F30001188E2050AD5302383F311884FF480619C
:103F4000281DFFF74DFF002383F311884FF0300940
:103F50004FF0000A14F0200838D13B0616D54FF078
:103F6000300905F1380A200610D589F3118850462A
:103F700000F07AF9002836DA0821281DFFF730FF13
:103F800027F080033360002383F31188790614D56A
:103F9000620612D5302383F31188D5E913239A42A0
:103FA00008D12B6C33B11021281D27F04007FFF7F3
:103FB00017FF3760002383F31188E30618D5AA6E34
:103FC0001369ABB1BDE8F0475069184789F3118810
:103FD000736A95F864102846194000F0E3F98AF3F3
:103FE0001188F469B6E7B06288F31188F469BAE71A
:103FF000BDE8F0874FF0E023002258684FF0FF3112
:10400000930003F1604303F5614301329042C3F82A
:104010008010C3F88011F3D27047000000F16043B4
:1040200003F561430901C9B283F80013012200F0CE
:104030001F039A4043099B0003F1604303F561436A
:10404000C3F880211A607047F8B515468268066982
:10405000AA420B46816938BF8568761AB542044684
:104060000BD218462A46FDF749FCA3692B44A361ED
:10407000A3685B1BA3602846F8BD0CD918463246DE
:10408000FDF73CFCAF1BE1683A463044FDF736FCD7
:10409000E3683B44EBE718462A46FDF72FFCE3684C
:1040A000E5E7000083689342F7B51546044638BF3C
:1040B0008568D0E90460361AB5420BD22A46FDF76E
:1040C0001DFC63692B446361A36828465B1BA360E6
:1040D00003B0F0BD0DD932460191FDF70FFC0199F7
:1040E000E068AF1B3A463144FDF708FCE3683B4407
:1040F000E9E72A46FDF702FCE368E4E710B50A4465
:104100000024C361029B8460C0E90000C0E905117E
:10411000C1600261036210BD08B5D0E90532934267
:1041200001D1826882B98268013282605A1C426180
:104130001970D0E904329A4224BFC3684361002158
:1041400000F078FA002008BD4FF0FF30FBE70000D8
:1041500070B5302304460E4683F31188A568A5B1D7
:10416000A368A269013BA360531CA361157822696F
:10417000934224BFE368A361E3690BB120469847EB
:10418000002383F31188284607E03146204600F0DB
:1041900041FA0028E2DA85F3118870BD2DE9F74F66
:1041A00004460E4617469846D0F81C904FF0300A49
:1041B0008AF311884FF0000B154665B12A46314647
:1041C0002046FFF741FF034660B94146204600F014
:1041D00021FA0028F1D0002383F31188781B03B063
:1041E000BDE8F08FB9F1000F03D001902046C84719
:1041F000019B8BF31188ED1A1E448AF31188DCE7CA
:10420000C0E90511C160C3611144009B8260C0E92F
:104210000000016103627047F8B504460D4616467A
:10422000302383F31188A768A7B1A368013BA3607B
:1042300063695A1C62611D70D4E904329A4224BF3A
:10424000E3686361E3690BB120469847002080F37F
:10425000118807E03146204600F0DCF90028E2DA58
:1042600087F31188F8BD0000D0E905239A4210B504
:1042700001D182687AB98268013282605A1C8261F7
:104280001C7803699A4224BFC3688361002100F04F
:10429000D1F9204610BD4FF0FF30FBE72DE9F74F75
:1042A00004460E4617469846D0F81C904FF0300A48
:1042B0008AF311884FF0000B154665B12A46314646
:1042C0002046FFF7EFFE034660B94146204600F066
:1042D000A1F90028F1D0002383F31188781B03B0E3
:1042E000BDE8F08FB9F1000F03D001902046C84718
:1042F000019B8BF31188ED1A1E448AF31188DCE7C9
:10430000026843681143016003B118477047000019
:104310001430FFF743BF00004FF0FF331430FFF7B6
:104320003DBF00003830FFF7B9BF00004FF0FF334A
:104330003830FFF7B3BF00001430FFF709BF0000AB
:104340004FF0FF311430FFF703BF00003830FFF7A4
:1043500063BF00004FF0FF323830FFF75DBF000051
:10436000012914BF6FF0130000207047FFF748BD0C
:10437000044B03600023C0E902334360012303744C
:10438000704700BF5054000810B53023044683F333
:104390001188FFF75FFD02232374002080F311884A
:1043A00010BD000038B5C36904460D461BB9042191
:1043B0000844FFF7A5FF294604F11400FFF7ACFEFF
:1043C000002806DA201D4FF40061BDE83840FFF7F1
:1043D00097BF38BD00230375826803691B6899681D
:1043E0009142FBD25A680360426010605860704787
:1043F00000230375826803691B6899689142FBD8A2
:104400005A680360426010605860704708B50846FB
:10441000302383F311880B7D032B05D0042B0DD0A3
:104420002BB983F3118808BD8B6900221A604FF005
:10443000FF338361FFF7CEFF0023F2E7D1E90032BB
:1044400013605A60F3E70000FFF7C4BF054BD9685B
:104450000875186802681A60536001220275D860F6
:10446000FCF7DAB81062002030B50C4BDD684B1C4D
:1044700087B004460FD02B46094A684600F06CF915
:104480002046FFF7E3FF009B13B1684600F06EF98A
:10449000A86907B030BDFFF7D9FFF9E71062002027
:1044A0000D440008044B1A68DB6890689B689842CA
:1044B00094BF00200120704710620020084B10B507
:1044C0001C68D86822681A60536001222275DC607B
:1044D000FFF78EFF01462046BDE81040FCF79CB870
:1044E00010620020044B1A68DB6892689B689A424D
:1044F00001D9FFF7E3BF70471062002038B5074CC1
:1045000007490848012300252370656000F030FC4E
:104510000223237085F3118838BD00BF7864002022
:104520007C5400081062002008B572B6044B186570
:1045300000F0E6FA00F09EFB024B03221A70FEE741
:10454000106200207864002000F046B9EFF311807B
:1045500020B9EFF30583302282F311887047000001
:1045600010B530B9EFF30584C4F3080414B180F337
:10457000118810BDFFF7B6FF84F31188F9E700003A
:104580008B60022308618B82084670478368A3F121
:10459000840243F8142C026943F8442C426943F81E
:1045A000402C094A43F8242CC26843F8182C0222F4
:1045B00003F80C2C002203F80B2C044A43F8102CAF
:1045C000A3F12000704700BF3106000810620020F0
:1045D00008B5FFF7DBFFBDE80840FFF735BF000077
:1045E000024BDB6898610F20FFF730BF106200209C
:1045F000302383F31188FFF7F3BF000008B50146AD
:10460000302383F311880820FFF72EFF002383F364
:10461000118808BD064BDB6839B1426818605A60E2
:10462000136043600420FFF71FBF4FF0FF30704757
:10463000106200200368984206D01A680260506039
:1046400099611846FFF700BF7047000010B5036876
:104650009C68A2420CD85C688A600B604C60216048
:10466000596099688A1A9A604FF0FF33836010BDD1
:104670001B68121BECE700000A2938BF0A2170B53D
:1046800004460D460A26601900F06CFB00F058FB4A
:10469000041BA54203D8751C2E460446F3E70A2ED8
:1046A00004D9BDE87040012000F0A2BB70BD00003D
:1046B000F8B5144B0D46D96103F1100141600A2A87
:1046C0001969826038BF0A22016048601861A81821
:1046D000144600F039FB0A2700F032FB431BA342CB
:1046E000064606D37C1C281900F03CFB27463546BD
:1046F000F2E70A2F04D9BDE8F840012000F078BBAA
:10470000F8BD00BF10620020F8B506460D4600F067
:1047100017FB0F4A134653F8107F9F4206D12A46D3
:1047200001463046BDE8F840FFF7C2BFD169BB681B
:10473000441A2C1928BF2C46A34202D92946FFF758
:104740009BFF224631460348BDE8F840FFF77EBF95
:10475000106200202062002010B4C0E9032300236F
:104760005DF8044B4361FFF7CFBF000010B5194C53
:10477000236998420DD0D0E90032816813605A60F5
:104780009A680A449A60002303604FF0FF33A361E4
:1047900010BD2346026843F8102F536000220260C8
:1047A00022699A4203D1BDE8104000F0D5BA93685F
:1047B00081680B44936000F0C3FA2269E169926852
:1047C000441AA242E4D91144BDE81040091AFFF787
:1047D00053BF00BF106200202DE9F047DFF8BC8016
:1047E00008F110072C4ED8F8105000F0A9FAD8F8AC
:1047F0001C40AA68031B9A423ED81444D5E90032F3
:104800004FF00009C8F81C4013605A60C5F80090CA
:10481000D8F81030B34201D100F09EFA89F3118824
:10482000D5E9033128469847302383F311886B6913
:10483000002BD8D000F084FA6A69A0EB04094A453D
:1048400082460DD2022000F0D3FA0022D8F81030B0
:10485000B34208D151462846BDE8F047FFF728BFCC
:10486000121A2244F2E712EB090938BF4A462946D8
:104870003846FFF7EBFEB5E7D8F81030B34208D062
:104880001444211AC8F81C00A960BDE8F047FFF7DE
:10489000F3BEBDE8F08700BF206200201062002058
:1048A00000207047FEE70000704700004FF0FF3027
:1048B00070470000BFF34F8F024A1369DB03FCD43B
:1048C000704700BF0020024008B5094B1B7873B940
:1048D000FFF7F0FF074B5A69002ABFBF064A9A60EC
:1048E00002F188329A601A6822F480621A6008BD68
:1048F00090640020002002402301674508B50B4B5F
:104900001B7893B9FFF7D6FF094B5A6942F0004272
:104910005A611A6842F480521A601A6822F480526E
:104920001A601A6842F480621A6008BD9064002020
:1049300000200240FF289ABF00F58030C00200200E
:10494000704700004FF40060704700004FF4807023
:1049500070470000FF2808B50BD8FFF7EBFF00F504
:1049600000630268013204D104308342F9D101208E
:1049700008BD0020FCE70000FF2838B5044626D813
:10498000FFF7E4FDFFF796FFFFF79EFF114BF322C1
:104990001A6102225A615A6942EAC4025A615A698A
:1049A00042F480325A6105462046FFF783FF4FF4F8
:1049B0000061FFF7BFFF00F059F92846FFF79EFF9F
:1049C000FFF7CEFD2046BDE83840FFF7C3BF00200B
:1049D00038BD00BF0020024040EA020313F0070385
:1049E0002DE9F04705460C46164606D0344B40F2FA
:1049F00031321A600020BDE8F0878118314A9142B7
:104A00000CD92F4A40F236311160F3E72B1D1B6899
:104A10006268934208D1083E08350834072E19D938
:104A20002A6823689A42F1D0FFF790FDFFF74CFF08
:104A3000FFF740FF04F10801234C4FF001084FF04D
:104A40000009012EA1F1080708D8FFF757FFFFF76B
:104A500087FD01E0002EE7D10120CCE7C4F81480E7
:104A6000AA4651F8083C4AF8043B51F8043C6B60F4
:104A7000FFF720FF236943F001032361C4F814907A
:104A80002A6851F8083C9A420ED00D4B40F25E3233
:104A90001A600E4B1D600E4B1E600E4B1F60FFF721
:104AA0002DFFFFF75DFDA5E7DAF800A051F8043C03
:104AB0009A4501F10801E8D1083E0835C1E700BF79
:104AC0008C64002000000808002002408064002060
:104AD0008864002084640020084908B50B7828B158
:104AE0001BB9FFF7F1FE01230B7008BD002BFCD0B2
:104AF000BDE808400870FFF701BF00BF90640020C8
:104B000008B54FF4C0314FF0005000F0B1F8BDE8E7
:104B100008404FF400414FF0805000F0A9B8000069
:104B2000084600F0F3BB000070B582B0FFF70EFD41
:104B30000E4E054600F004F93268904237BF0C4A29
:104B40000B49516814682EBFD1E900410131516011
:104B50000419034641F10001284601913360FFF733
:104B6000FFFC0199204602B070BD00BF9464002094
:104B70009864002070B582B0FFF7E8FC104E05463F
:104B800000F0DEF83268904237BF0E4A0D49516896
:104B900014682EBFD1E9004101315160041941F17F
:104BA00000010346284601913360FFF7D9FC0199C3
:104BB0004FF47A7200232046FBF71AFB02B070BD57
:104BC00094640020986400200244D2B2904200D144
:104BD0007047431C800000F1804000F514500068CD
:104BE00041F8040BD8B2F1E7124B10B5D3F890405E
:104BF000240409D4D3F89040C3F89040D3F89040EF
:104C000044F40044C3F890400B4C2368024443F43E
:104C100080732360D2B2904200D110BD431C80004B
:104C200000F1804000F5145051F8044B0460D8B2F4
:104C3000F1E700BF001002400070004007B50122FC
:104C400001A90020FFF7C0FF019803B05DF804FB45
:104C500013B50446FFF7F2FFA04205D0012201A9D7
:104C600000200194FFF7C0FF02B010BD70470000A4
:104C70007047000070470000074B45F255521A601C
:104C800002225A6040F6FF729A604CF6CC421A60DB
:104C9000024B01221A70704700300040A4640020CB
:104CA000034B1B781BB1034B4AF6AA221A607047CC
:104CB000A464002000300040054B1A6832B902F1AC
:104CC000804202F50432D2F894201A60704700BF87
:104CD000A0640020024B4FF40002C3F894207047F8
:104CE0000010024008B5FFF7E7FF024B1868C0F359
:104CF000407008BDA064002070470000FEE700007F
:104D00000A4B0B480B4A90420BD30B4BDA1C121A7E
:104D1000C11E22F003028B4238BF00220021FCF7A3
:104D2000FFBD53F8041B40F8041BECE7EC550008EA
:104D300028650020286500202865002000F0C2B802
:104D40004FF08043586A70474FF080430022586309
:104D50001A610222DA6070474FF080430022DA6065
:104D6000704700004FF0804358637047FEE7000033
:104D700070B51B4B01630025044686B05860856200
:104D80000E46FEF7DFFF04F11003C4E904334FF0D1
:104D9000FF33C4E90635C4E90044A560E562FFF7C6
:104DA000CFFF2B460246C4E9082304F134010D4A23
:104DB000256580232046FFF7E3FB0123E0600A4AD4
:104DC0000375009272680192B268CDE90223074B25
:104DD0006846CDE90435FFF7FBFB06B070BD00BFA8
:104DE00078640020885400088D5400086D4D000838
:104DF000024AD36A1843D062704700BF1062002095
:104E00004B6843608B688360CB68C3600B69436108
:104E10004B6903628B6943620B6803607047000053
:104E200008B5204BDA6A42F07F02DA62DA6A22F0D1
:104E30007F02DA62DA6ADA6C42F07F02DA64DA6EF2
:104E400042F07F02DA66184ADB6E11464FF090405E
:104E5000FFF7D6FF02F11C0100F58060FFF7D0FFDD
:104E600002F1380100F58060FFF7CAFF02F154013A
:104E700000F58060FFF7C4FF02F1700100F580606B
:104E8000FFF7BEFF02F18C0100F58060FFF7B8FF6D
:104E900002F1A80100F58060FFF7B2FFBDE808400D
:104EA00000F050B8001002409454000808B500F01B
:104EB000FBF9FFF723FBBDE80840FFF7FDBE00004C
:104EC000704700000F4B9A6D42F001029A659A6F8D
:104ED00042F001029A670C4A9B6F936843F001030A
:104EE00093604FF08043A7229A624FF0FF32DA625C
:104EF00000229A615A63DA605A6001225A611A608C
:104F0000704700BF00100240002004E04FF08042D4
:104F100008B51169D3680B40D9B2C9439B07116129
:104F200007D5302383F31188FFF70EFB002383F3AB
:104F3000118808BD08B5FFF75DF8BDE8084000F02E
:104F40008BB900004E4B4FF0FF319A6A99629A6A12
:104F500000229A62986AD86A60F07F00D862D86AA4
:104F600000F07F00D862D86A186B1963186B1A6357
:104F7000186B986B9963986B9A63986BD86BD9632D
:104F8000D86BDA63D86B186C1964196C1A64196CD5
:104F9000196E41F001011966D3F8801021F001016A
:104FA000C3F88010D3F88010996D41F08051996555
:104FB000996F21F080519967996F32494FF4004001
:104FC0008860CA600A624A628A62CA620A634A6385
:104FD0008A63CA630A644A648A64CA640A654A6561
:104FE0004A604FF48072C1F880204FF440720A602A
:104FF0004A6912F48062FBD1D3F8901011F4407F1B
:105000001EBF4FF48031C3F89010C3F89020D3F83E
:10501000982042F00102C3F89820D3F89820920714
:10502000FBD51A6842F480321A601A689003FCD5E6
:10503000D3F8902022F00322C3F89020124ADA60BD
:105040001A6842F080721A601A689101FCD50F4903
:105050000F4800229A60C3F888100E49C3F89C20BC
:10506000016002684A401207FBD19A6842F00302CD
:105070009A609A6802F00C020C2AFAD1704700BFBD
:105080000010024000700040132A610155010050D9
:105090000020024004070400074A08B5536903F0E2
:1050A0000103536123B1054A13680BB15068984757
:1050B000BDE80840FEF76ABE00040140A864002075
:1050C000074A08B5536903F00203536123B1054A47
:1050D00093680BB1D0689847BDE80840FEF756BE0C
:1050E00000040140A8640020074A08B5536903F092
:1050F0000403536123B1054A13690BB15069984702
:10510000BDE80840FEF742BE00040140A86400204C
:10511000074A08B5536903F00803536123B1054AF0
:1051200093690BB1D0699847BDE80840FEF72EBEE1
:1051300000040140A8640020074A08B5536903F041
:105140001003536123B1054A136A0BB1506A9847A3
:10515000BDE80840FEF71ABE00040140A864002024
:10516000164B10B55C6904F478725A61A30604D535
:10517000134A936A0BB1D06A9847600604D5104A67
:10518000136B0BB1506B9847210604D50C4A936BF7
:105190000BB1D06B9847E20504D5094A136C0BB1EB
:1051A000506C9847A30504D5054A936C0BB1D06C9D
:1051B0009847BDE81040FEF7E9BD00BF000401407C
:1051C000A8640020194B10B55C6904F47C425A6154
:1051D000620504D5164A136D0BB1506D984723052F
:1051E00004D5134A936D0BB1D06D9847E00404D5F4
:1051F0000F4A136E0BB1506E9847A10404D50C4AA8
:10520000936E0BB1D06E9847620404D5084A136FB1
:105210000BB1506F9847230404D5054A936F0BB127
:10522000D06F9847BDE81040FEF7B0BD00040140C4
:10523000A864002008B50348FEF758FEBDE8084002
:10524000FEF7A4BDA05F002008B5FFF75FFEBDE834
:105250000840FEF79BBD0000062108B50846FEF792
:10526000DDFE06210720FEF7D9FE06210820FEF705
:10527000D5FE06210920FEF7D1FE06210A20FEF701
:10528000CDFE06211720FEF7C9FE06212820FEF7D5
:10529000C5FE07211C20FEF7C1FEBDE808400C2119
:1052A0002620FEF7BBBE000008B5FFF743FE00F066
:1052B00009F8FFF75BF8FFF703FEBDE80840FFF7CA
:1052C0003DBD00000023054A19460133102BC2E9F9
:1052D000001102F10802F8D1704700BFA864002055
:1052E0000B460146184600F003B8000000F00EB867
:1052F00010B5054C13462CB10A4601460220AFF307
:10530000008010BD2046FCE700000000024B014673
:105310001868FFF705BC00BF2823002010B501392D
:105320000244904201D1002005E0037811F8014FBA
:10533000A34201D0181B10BD0130F2E72DE9F04166
:10534000A3B1C91A17780144044603F1FF3C8C420B
:10535000204601D9002009E00578BD4204F101048E
:10536000F5D10CEB0405D618A54201D1BDE8F081BA
:1053700015F8018D16F801EDF045F5D0E7E70000CE
:10538000034611F8012B03F8012B002AF9D17047CD
:105390006F72672E6172647570696C6F742E486FDE
:1053A0006C7962726F47345F4750530053544D33EA
:1053B0003247343F3F00000040A2E4F164689106A8
:1053C0000041A3E5F2656992070000004261642094
:1053D00043414E496661636520696E6465782E00BD
:1053E000000100000001FF00006400400068004070
:1053F0000000000000000000ED240008C91F0008A4
:10540000052C0008C11F0008712000085522000863
:10541000392000080120000805200008DD1F0008D1
:10542000C51F000815220008E91F0008712D00089B
:10543000F51F0008E92100080096000000000000A8
:10544000000000000000000000000000000000005C
:10545000000000002D4300081943000855430008D0
:10546000414300084D430008394300082543000824
:1054700011430008614300086330000078540008BD
:1054800068620020786400206D61696E0069646C58
:1054900065000000A000802A00000000AAAAAAAAB5
:1054A00050000024FFFF000000770000009009007A
:1054B0000400005A00000000AAAAAA9A04000000F2
:1054C000FFBF000000000000000099000011101450
:1054D00000000000AAAAAAA600010010FFDF000039
:1054E00000000000000000000000000000000000BC
:1054F000AAAAAAAA00000000FFFF00000000000006
:10550000000000000000000000000000AAAAAAAAF3
:1055100000000000FFFF000000000000000000008D
:105520000000000000000000AAAAAAAA00000000D3
:10553000FFFF00000000000000000000000000006D
:1055400000000000AAAAAAAA00000000FFFF0000B5
:105550000000000000000000C8ACFF7F0100000058
:105560001D040000000000000070070000000000A3
:10557000FE2A0100D2040000FF000000A05F00200E
:1055800000000000AC5300082C23002000000000A5
:10559000000000000000000000000000000000000B
:1055A00000000000000000000000000000000000FB
:1055B00000000000000000000000000000000000EB
:1055C00000000000000000000000000000000000DB
:1055D00000000000000000000000000000000000CB
:0C55E000000000000000000000000000BF
:00000001FF
